:1000000012C02CC02BC02AC029C028C027C026C0BF
:1000100025C024C023C022C021C020C01FC01EC0D4
:100020001DC0C7C01BC011241FBECFE5D4E0DEBF7A
:10003000CDBF10E0A0E6B0E0E2ECF2E002C0059037
:100040000D92AE36B107D9F710E0AEE6B0E001C0D0
:100050001D92A037B107E1F702D031C1D1CFCF93C4
:1000600014BE88E10FB6F89481BD11BC0FBE86E0C6
:1000700087BB8CE084BB11BA82E4EFD02ED03DD098
:1000800078942DE088E190E00FB6F894A89581BDB2
:100090000FBE21BD80E690E0E9D0C4E0F5D0882312
:1000A00029F088B38C2788BB5FD0E0D0A895F6CF25
:1000B00097B1907F97B997B18F70892B87B9369A8E
:1000C000089581E0369980E00895FBDF8823E9F305
:1000D000369824B135B1C901089517B83E9A86B152
:1000E000856086B9379A80E0E3DFEFDF0895EDDFC2
:1000F00096958795969587950895AB9AAA980895B1
:1001000081E0D6DFF4DF08950F931F93CF93DF9341
:10011000D82FC92FF5DF90E08C599F4F6AE070E02F
:10012000BAD09B01CE01E92FF82F10E0CAE0D0E051
:100130000FEF408150E0249FC001259F900D349F18
:10014000900D1124BE01A7D06F3F710519F010F07A
:10015000008301C060831F5F3196173051F7DF9134
:10016000CF911F910F910895CF93DF93AB988FE1BB
:1001700091E00197F1F700C00000C0E6D0E0AA9A34
:1001800095E69A95F1F70000AA9880EC8A95F1F728
:1001900080E08EDFACDF899390E0C736D90779F72E
:1001A000AB9ACE010797B0DFCE010797DF91CF91D1
:1001B00008951F920F920FB60F9211248F939F9361
:1001C000EF93FF9381B190E0887F883B9105C1F068
:1001D000893B91053CF4883A910559F0803B9105A3
:1001E00081F507C0803C910531F1883C910549F5C6
:1001F00022C081E080936F008091670083B915C0B1
:1002000080916F00863040F010926F0080916D00F9
:1002100083B986B78F7B11C0E82FF0E0E959FF4F13
:10022000908193B98F5F80936F0086B7806486BF9B
:1002300010926E0006C086B7806486BF81E080930E
:100240006E0086B7806886BFFF91EF919F918F9176
:100250000F900FBE0F901F901895882311F481E026
:1002600001C08E7F82B985E486BF0895282F392F7B
:10027000D901E7E6F0E08D91819380E0EE36F80752
:10028000D1F710926E00089581E090916E0099234D
:1002900009F480E00895AA1BBB1B51E107C0AA1F07
:1002A000BB1FA617B70710F0A61BB70B881F991F17
:1002B0005A95A9F780959095BC01CD010895F894C1
:0202C000FFCF6E
:0E02C2008080808080808042424242424242E0
:00000001FF
